:1000000028288F018E00FF308E07031C8F07031CEA
:10001000232803308D00DF300F2003288D01E83EB8
:100020008C008D09FC30031C18288C070318152838
:100030008C0764008D0F15280C181E288C1C222894
:1000400000002228080083130313831264000800B1
:100050008316850186018312051583160511831207
:10006000851183168511831201308F00F430022030
:1000700005118316051183128515831685118312C8
:0E00800001308F00F43002202C286300452848
:02400E00FD3F74
:00000001FF
